:100000000CC0189518951895189596C08EC018951F
:10001000189518951895AAAAAAAA0FED0DBF479A88
:100020000FEF07BB00E008BB00E001BB0EE702BB1F
:100030000EEF02BB01E003BF02E009BF03E00EBD0B
:1000400002E809BF00E00CBD0DBDF0E0EDE1F0837A
:10005000EA95E9F778946130F1F700E00EBD60E0D1
:100060006EBBE09A2DB3A0E100C038C067D052D07B
:100070002F793A1741F54F734C3089F0C09B21C05E
:10008000403071F0413069F0423061F0433059F056
:10009000403151F0413149F070E0872F12C096C0D5
:1000A000A7C0A9C0ABC0ADC0AFC0B0C0842FDDCF6A
:1000B000E199FECF60E02DBB6EBBF894E29AE19A25
:1000C000789428BBD2CF70E0872F28BBCECFC4E175
:1000D000DFEFDA95F1F7CA95D9F70895D0B3DE735B
:1000E000CCE3CD1769F0CAE3CD1761F0C6E3CD17B5
:1000F00059F0CEE2CD1751F0CEE1CD1749F0B6CF91
:100100004CE0BACF40E0B8CF41E0B6CF42E0B4CF48
:1001100043E0B2CFC09B0895DADFE395D6E9ED174F
:1001200009F00895C79A206808950FB6139513949F
:1001300009F403950FBE18956395189511240027AF
:100140001127083008F03FC017331CF4809BF8CF0C
:10015000F8CF0830C4F58099FCCF112711319CF5F8
:10016000809BFCCF012F1127202E2694322C200EAD
:10017000000F300E12153CF58099FCCF11275CE082
:10018000442733271215F0F3809909C08894441F3F
:10019000331F1315C4F4809BFCCF112708C00894AB
:1001A000441F331F13157CF48099FCCF11275A95F7
:1001B00049F7042F001F331F001F331F35FB46F97B
:1001C0004F773F710895442733270895682F6417A8
:1001D00049F4703039F471E020FF05C02E7FB22F52
:1001E000222766CF63CFBF77EE272B2F216060CF0A
:1001F000217E226066CF217E246063CF217E28602D
:1002000060CF217E20615DCF20625BCF206459CF1B
:04021000206857CF3C
:00000001FF
